:100000000C9461000C947E000C947E000C947E0095
:100010000C947E000C947E000C947E000C947E0068
:100020000C947E000C947E000C947E000C947E0058
:100030000C947E000C947E000C947E000C947E0048
:100040000C949A000C947E000C947E000C947E001C
:100050000C947E000C947E000C947E000C947E0028
:100060000C947E000C947E00000000002400270009
:100070002A0000000000250028002B0000000000DE
:1000800023002600290004040404040404040202DA
:100090000202020203030303030301020408102007
:1000A0004080010204081020010204081020000012
:1000B0000007000201000003040600000000000029
:1000C000000011241FBECFEFD4E0DEBFCDBF11E092
:1000D000A0E0B1E0EAE3F4E002C005900D92A030A8
:1000E000B107D9F711E0A0E0B1E001C01D92A9303D
:1000F000B107E1F70E940A020C941B020C94000065
:100100008DE061E00E94B50168EE73E080E090E070
:100110000E94E2008DE060E00E94B50168EE73E0AD
:1001200080E090E00E94E20008958DE061E00E948E
:10013000760108951F920F920FB60F9211242F93FC
:100140003F938F939F93AF93BF93809104019091BE
:100150000501A0910601B0910701309108010196B7
:10016000A11DB11D232F2D5F2D3720F02D57019696
:10017000A11DB11D209308018093040190930501F6
:10018000A0930601B09307018091000190910101B5
:10019000A0910201B09103010196A11DB11D8093B0
:1001A000000190930101A0930201B0930301BF915C
:1001B000AF919F918F913F912F910F900FBE0F9014
:1001C0001F9018959B01AC017FB7F89480910001B6
:1001D00090910101A0910201B091030166B5A89B25
:1001E00005C06F3F19F00196A11DB11D7FBFBA2F49
:1001F000A92F982F8827860F911DA11DB11D62E0A0
:10020000880F991FAA1FBB1F6A95D1F7BC012DC08B
:10021000FFB7F8948091000190910101A091020133
:10022000B0910301E6B5A89B05C0EF3F19F0019618
:10023000A11DB11DFFBFBA2FA92F982F88278E0FA0
:10024000911DA11DB11DE2E0880F991FAA1FBB1FC0
:10025000EA95D1F7861B970B885E9340C8F2215030
:1002600030404040504068517C4F211531054105D8
:10027000510571F60895789484B5826084BD84B583
:10028000816084BD85B5826085BD85B5816085BD91
:10029000EEE6F0E0808181608083E1E8F0E01082AA
:1002A000808182608083808181608083E0E8F0E0EB
:1002B000808181608083E1EBF0E0808184608083D5
:1002C000E0EBF0E0808181608083EAE7F0E080810C
:1002D000846080838081826080838081816080836C
:1002E0008081806880831092C1000895CF93DF934E
:1002F000482F50E0CA0186569F4FFC0134914A575F
:100300005F4FFA018491882369F190E0880F991F6B
:10031000FC01E859FF4FA591B491FC01EE58FF4F45
:10032000C591D491662351F42FB7F8948C91932FF3
:10033000909589238C93888189230BC0623061F466
:100340002FB7F8948C91932F909589238C93888163
:10035000832B88832FBF06C09FB7F8948C91832B83
:100360008C939FBFDF91CF910895482F50E0CA0131
:1003700082559F4FFC012491CA0186569F4FFC0174
:1003800094914A575F4FFA013491332309F440C0E6
:10039000222351F1233071F0243028F42130A1F0D0
:1003A000223011F514C02630B1F02730C1F02430CE
:1003B000D9F404C0809180008F7703C080918000C1
:1003C0008F7D8093800010C084B58F7702C084B584
:1003D0008F7D84BD09C08091B0008F7703C080916C
:1003E000B0008F7D8093B000E32FF0E0EE0FFF1F91
:1003F000EE58FF4FA591B4912FB7F894662321F4DE
:100400008C919095892302C08C91892B8C932FBF5E
:1004100008950895CF93DF930E943B010E94090243
:100420000E949500C0E0D0E00E9480002097E1F398
:0A0430000E940000F9CFF894FFCFFE
:00000001FF
